:020000040800F2
:100000006009002045010008051100086D10000876
:1000100001110008CD0100084F2F0008000000006A
:100020000000000000000000000000001126000891
:10003000FD0D000800000000B12100085D28000847
:100040005F0100085F0100085F0100085F01000810
:100050005F0100085F0100085F0100085F01000800
:100060005F0100085F0100085F0100085F010008F0
:100070005F0100085F0100085F0100085F010008E0
:100080005F0100085F0100085F0100085F010008D0
:100090005F0100085F0100085F0100085F010008C0
:1000A0005F0100085F0100085F0100085F010008B0
:1000B0005F010008C52800085F0100085F01000813
:1000C0005F0100085F0100085F0100085F01000890
:1000D0005F010008A52A0008012B0008E52B000895
:1000E0005F0100085F0100085F0100085F01000870
:1000F0005F0100085F0100085F0100085F01000860
:100100005F0100085F0100085F0100085F0100084F
:100110005F0100085F0100085F0100085F0100083F
:100120005F0100085F0100085F0100085F0100082F
:10013000DFF80CD000F038F80048004755300008D0
:10014000600900200648804706480047FEE7FEE7B2
:10015000FEE7FEE7FEE7FEE7FEE7FEE7FEE7FEE777
:100160006128000831010008D2B201E000F8012B3B
:10017000491EFBD270470022F6E710B513460A4627
:1001800004461946FFF7F0FF204610BD30B504467F
:100190000020034600E05B1C934203D2E05CCD5C90
:1001A000401BF8D030BD0000064C074D06E0E0686B
:1001B00040F0010394E8070098471034AC42F6D3AE
:1001C000FFF7BAFFAC330008CC33000800BFFEE7EE
:1001D00010B502460B460020002104E0545C0444A4
:1001E000E0B24C1CE1B29942F8DBC443E0B2441CDB
:1001F000E0B210BDFEB5002000900190029000F02A
:100200004FFF404800780A2822D13F4800783F49F4
:100210000978884218D13C4840783C49497888425E
:1002200012D13948007A3949097A88420CD13648C6
:10023000407A3649497A884206D13548008840F4E8
:1002400000403349088003E014212F48FFF793FF53
:100250002F48008800F40040002852D02D4800218B
:10026000016001712C48016001712C48016001712D
:100270002B4801600171002027490870224800794D
:1002800048702148407988701F488079C8701E489E
:10029000C0790871052223491F48FFF777FFA0B1F5
:1002A0000020214908701C48407848701A4880781E
:1002B00088701948C078C8701748007908711948C3
:1002C00015490A68026009790171134840780406EB
:1002D0001148807805041048C0780602601930443F
:1002E0000D490979471801201049087000F0D8FE1F
:1002F0000020044908700649088014210248FFF7CD
:100300003AFFFEBD09000020D40100200C000020AF
:100310000A00002032000020160000203A000020D1
:100320003F000020200000201B000020470000208C
:1003300010B588B07F480078012838D100207D4969
:100340000870FC207C490870112048707B480078B8
:1003500088707A484078C870784880780871774803
:10036000C078487175480079887107217248FFF795
:100370002FFF7149C871002071490860FF22E121F7
:10038000012001F063FE08236B4AA821012001F03F
:100390001FFE012001F0A2F901206A49C1F8A40161
:1003A0006949087000206949088000F079FE6748B3
:1003B000008840F6B83188427BDC00F071FE60486E
:1003C00084380068002857D100F06AFE6946012091
:1003D00001F0DCFD0446204602F068F95CA002F062
:1003E0006FF904F040004028EDD100208DF80A009C
:1003F0000721684600F003FD55A002F061F99DF861
:1004000001004E490978884254D19DF802004B49B9
:10041000497888424ED19DF803004849897888423E
:1004200048D19DF804004549C978884242D19DF8D9
:1004300005004249097988423CD1434800780128A7
:100440001BD141480078401C3F49087012203A49AE
:10045000487007213848FFF7BBFE3749C8710020B4
:10046000374908600823344AA821012001F0B0FD73
:1004700001203449C1F8A40158E000203249087035
:100480000E21344800F0BBFC31A002F019F93248CB
:100490000178012001F07CF910202E4948700E21CE
:1004A0002C4802F0F7F82DA002F00AF9012008B05C
:1004B00010BD16E000202249086011201E49487036
:1004C00007211D48FFF784FE1B49C87108230A460F
:1004D000A821012001F07CFD01201A49C1F8A401E6
:1004E00024E000201549087048708870C8700871B1
:1004F0001B49087048708870C870087119490870E5
:1005000048708870C8700871174908704870887002
:10051000C870087130200F4948700E210D4802F054
:10052000B9F812A002F0CCF80120C0E700F0B8FD45
:100530000020BCE7440000204800002032000020DA
:10054000A481214200802142880000202600002052
:100550000A000000C8030020300000204F4B0A00B2
:100560003F0000201B0000201600002033303030F8
:100570000A00000010B588B04B480088B0F5FA6F4B
:1005800071DA4A48006800286ED100F089FD69469A
:10059000012001F0FBFC044604F04000402875D126
:1005A00000208DF80A009DF8010078B99DF802003E
:1005B00060B99DF8030048B900203D4908704870B3
:1005C0008870C8700871012008B010BD39480078E3
:1005D000072803D0374800780D280FD10020344970
:1005E00008709DF8000048709DF8010088709DF823
:1005F0000200C8709DF80300087145E02D4800789E
:10060000082810D19DF80100294908709DF80200C2
:1006100048709DF8030088709DF80400C8709DF82C
:100620000500087130E023480078092803D02148EC
:1006300000780E2819D100201D4908709DF801008E
:1006400080F0530048709DF8020080F043008870ED
:100650009DF8030080F04400C8709DF8040080F00D
:100660005800087110E014E010E0002010490870F4
:100670009DF8010048709DF8020088709DF8030005
:10068000C8709DF80400087101209DE700F008FD86
:1006900008E000200649087048708870C87008712A
:1006A000012091E700208FE73800002020812142BF
:1006B0003F0000203000002010B500F0F1FCFE48A3
:1006C0000078082829D1FD480078752825D1FB48F5
:1006D0004078702821D1F948807864281DD1F748E6
:1006E000C078612819D1F5480079742815D1F348EC
:1006F0004079652811D10020EF49087000BFF0480B
:10070000006800F4E060EF490843001DEC49086010
:10071000BFF34F8F00BF00BFFEE7E84800787528A1
:1007200007D0E6480078FA2803D00020E249087094
:1007300010BDE14800780E2800DAF9E7DE480078BD
:10074000401EDE49085CFB2800D0F1E7DB48807AD8
:10075000A02804D1D8480078152800D0E8E7D6486A
:1007600000780E281ED1D5480078FA2814D1D34835
:10077000407BFB2810D1D448008840F40040D24987
:1007800008800020CC4908700E21CC4800F037FBCF
:10079000CEA001F095FF4AE00020C7490870CA4981
:1007A000088044E0C448007815281ED1C34800786A
:1007B000FA2814D1C148007DFB2810D1C248008816
:1007C00040F40040C04908800020BB490870152152
:1007D000BA4800F014FBBDA001F072FF27E0002032
:1007E000B5490870B849088021E0B348007811285D
:1007F0001DD1B2480078FA2814D1B048007CFB28FB
:1008000010D1B148008840F40040AF490880002072
:10081000A94908701121A94800F0F1FAABA001F034
:100820004FFF04E00020A4490870A7490880A648AB
:10083000008800F40040002871D000F031FC9F488F
:100840008079A34988719D48C179A148C1719B48AD
:10085000017A9F4801729948417A9D4841729748B0
:10086000807A9B498872084680799A4988719848AD
:10087000C1799848C1719648017A964801729448A6
:10088000417A944841729248807A94284CD018DC7E
:10089000732834D00CDC252825D004DC21281AD07C
:1008A00022287DD11BE0262821D07128F9D122E011
:1008B000742828D075282AD078282CD08228F0D106
:1008C0002EE0A03809286BD2DFE800F0329CA0F5BA
:1008D000F4F3F2F1F00000207D498872CBE10020B2
:1008E0007B498872C7E1002079498872C3E1002002
:1008F00077498872BFE1002075498872BBE100200A
:1009000073498872B7E1002071498872B3E1002011
:100910006F498872AFE100206D498872ABE1AEE1AA
:1009200000206B498872A6E1002069498872A2E123
:100930000020614908706648807967498871644879
:10094000C1796548C1716248017A634801726048A3
:10095000417A614841725E48807A5F49887257489F
:10096000407B5B4948735548817B594881735348A4
:10097000C17B5748C1735148017C554801744F48A9
:10098000417C534841744D48407B544908704B4862
:10099000807B48704948C07B88704848007C00E0F4
:1009A00068E1C8704548407C087101204C490870D6
:1009B00000204C490880012000F090FE4AA001F080
:1009C0007FFE04E0FFF7B4FC044604B100E0F9E761
:1009D00000BF45A001F074FE002045490870487032
:1009E0008870C87008714349087048708870C87072
:1009F00008714149087048708870C870087134499E
:100A0000887238E100203249887234E139484078F0
:100A100048B93848807830B93648C07818B9354870
:100A2000007900B927E1002023490870284880791F
:100A3000324988712648C1793048C1712448017A09
:100A40002E4801722248417A2C4841722048807A0F
:100A50002A4988720120C872062008730020487352
:100A60002448017825488173224841782348C1737E
:100A700020488178214801741E48C1781F4841747C
:100A80001C4801791D488174162101F003FE3220B3
:100A900002F08CFA1621194800F0B1F90BA001F010
:100AA0000FFE002013490870487029E099E0DDE04E
:100AB000D8E0D3E02BE029E0030000200C01002067
:100AC0000CED00E00000FA05040000200A00000020
:100AD000000300209C020020C803002032000020F8
:100AE0004400002026000020303030300A00000092
:100AF0003F0000201B00002016000020640300209F
:100B00008870C87008715F498872B4E0B3E0002053
:100B10005D4908705D480178012000F039FE002031
:100B20005B4908805BA001F0CBFD04E0FFF722FDEC
:100B3000044604B100E0F9E700BF56A001F0C0FD93
:100B400050488079554988714E48C1795348C171E0
:100B50004C48017A514801724A48417A4F484172E3
:100B60004848807A4D4988720120C872062008736F
:100B7000002048734A4801784848817348484178C2
:100B80004648C17346488178444801744448C17856
:100B9000424841744248017940488174162101F06D
:100BA00079FD322002F002FA16213C4800F027F9C4
:100BB00039A001F085FD002039490870487088701F
:100BC000C87008713749087048708870C87008711B
:100BD0003549087048708870C87008712949887252
:100BE00049E03248407B29490870264880793049DD
:100BF00088712448C1792E48C1712248017A2C4855
:100C000001722048417A2A4841721E48807A284958
:100C10008872012048700E21254801F03BFD3220EA
:100C200002F0C4F9194800782249088001F0FAFC62
:100C300000201B49087048708870C87008711949F5
:100C4000087048708870C87008711749087048703B
:100C50008870C87008710B4988720CE0002009493F
:100C6000887208E000200749887204E000200549E6
:100C7000887200E000BF00BF00200F49088000BF5D
:100C800056E5000000030020030000203000002093
:100C900038000020343434340A000000640300209B
:100CA0003F0000201B000020160000200C01002047
:100CB0002C0400203405002004000020FA204A49BA
:100CC0000870102048700020887000214648C170CC
:100CD0000171417100204449887100214248C1716D
:100CE0000172417200204049C87400213E480175DC
:100CF000FB203D494875FA203C4908701020487097
:100D00000020887000213948C170017141710020B4
:100D10003649887100213548C17101724172002045
:100D2000324981F84B000021304880F84C10FB20FC
:100D30002E4981F84D00FA202D4908701020487086
:100D40000020887000212A48C17001714171002083
:100D50002749887100212648C17101724172002023
:100D60002349C872002122480173FB20204948739F
:100D7000FA20204908701020487000208870002157
:100D80001C48C1700171417100201A49887100210D
:100D90001848C1710172417200201649C8740021BF
:100DA00014480175FB2013494875FA201249087050
:100DB000102048700020887000210F48C170017118
:100DC000417100200C49887100210B48C1710172EA
:100DD000417200200849C872002107480173FB20B6
:100DE00005494873704700009C0200200003002062
:100DF0002C04002064030020C803002070472DE964
:100E0000F04104460E460DE02578281100F030F937
:100E1000074601F04BFC284600F02AF9074601F08E
:100E200045FC641C301EA6F10101CEB2ECD1BDE838
:100E3000F081000030B5044604254FF4302000F066
:100E40006FF80546042D17D10C48006940F00200E8
:100E50000A49086108464461006940F040000861A1
:100E60004FF4302000F05CF805460448006941F674
:100E7000FD71084001490861284630BD002002404C
:100E800004200B49C96801F0010109B101200EE0FD
:100E90000749C96801F0040109B1022007E00449CB
:100EA000C96801F0100109B1032000E00420704777
:100EB000002002400348006940F0800001490861B9
:100EC000704700000020024070B504460D4604261D
:100ED000F00200F025F80646042E11D109480069F9
:100EE00040F00100074908612580F00200F018F881
:100EF00006460448006941F6FE7108400149086150
:100F0000304670BD00200240024803494860034853
:100F1000486070472301674500200240AB89EFCD50
:100F200000B502460423FFF7ABFF034603E0FFF7DB
:100F3000A7FF0346521E012B01D1002AF7D102B9A7
:100F40000523184600BD2DE9F04102460025002684
:100F5000002000230024002791F803C00CF00F05A7
:100F600091F803C00CF0100CBCF1000F03D091F805
:100F700002C04CEA050591F800C0BCF1000F31D069
:100F8000146800202BE04FF0010C0CFA00F3B1F8CC
:100F900000C00CEA03069E4220D183004FF00F0CE4
:100FA0000CFA03F7BC4305FA03FC4CEA040491F87D
:100FB00003C0BCF1280F06D14FF0010C0CFA00FC65
:100FC000C2F814C00AE091F803C0BCF1480F05D183
:100FD0004FF0010C0CFA00FCC2F810C0401C0828AD
:100FE000D1D31460B1F800C0BCF1FF0F34DD5468F8
:100FF00000202EE000F1080C4FF0010808FA0CF375
:10100000B1F800C00CEA03069E4221D183004FF0E4
:101010000F0C0CFA03F7BC4305FA03FC4CEA04047A
:1010200091F803C0BCF1280F05D100F1080C08FAB3
:101030000CF8C2F8148091F803C0BCF1480F07D136
:1010400000F1080C4FF0010808FA0CF8C2F8108003
:10105000401C0828CED35460BDE8F0814161704740
:101060000161704701460A8890B2704700BFFEE7F1
:101070000146002001F00F02092A04DC01F00F02F2
:1010800002F1300003E001F00F023732D0B27047B6
:101090004CF6CC4001490860704700000030004029
:1010A00010B500F013F810BD70B505460C4645F2BA
:1010B000555000F01FF8284600F010F8204600F0C8
:1010C00013F800F003F8FFF7E3FF70BD4AF6AA201B
:1010D0000149086070470000003000400149486045
:1010E00070470000003000400149886070470000F0
:1010F00000300040014908607047000000300040A7
:1011000000BFFEE7704700007CB5054612A103C989
:10111000CDE900010821284601F052FA05236A466C
:101120003021284600F054FF05236A461021284646
:1011300000F0BEFE002406E01DF80400A52800D043
:1011400003E0601CC4B2052CF6DB00BF052C01D007
:1011500001207CBD0020FCE7A5A5A5A5A5000000F9
:1011600008B501211C2001F035F84020ADF8000041
:1011700010208DF8030003208DF8020069463248E4
:10118000FFF7E1FE40213048FFF76AFF1020ADF87D
:10119000000069462D48FFF7D6FE10212B48FFF7C7
:1011A0005FFF8020ADF8000048208DF80300032089
:1011B0008DF8020069462448FFF7C5FE4FF4007021
:1011C000ADF8000010208DF8030003208DF8020018
:1011D00069461D48FFF7B7FE4FF400711A48FFF744
:1011E0003FFF4FF48050ADF8000069461648FFF706
:1011F000AAFE4FF480511448FFF732FF4FF480707D
:10120000ADF8000048208DF8030003208DF802009F
:1012100069460D48FFF797FE01F000F901F0BCF8B0
:1012200000200B49086001200A49C1F89001002004
:1012300007490C31086001200749C1F8B0010821B5
:10124000002001F0BDF908BD000C0140000801407C
:1012500098812142000021420080214210B50446BD
:1012600002222321204600F0F1FE05231E4A2A21F6
:10127000204600F0ADFE05231B4A3021204600F039
:10128000A7FE3F222121204600F0E0FE012222217C
:10129000204600F0DBFE1A222521204600F0D6FE73
:1012A00024222621204600F0D1FE0F2220212046B4
:1012B00000F0CCFE0A223121204600F0C7FE0122B8
:1012C0003D21204600F0C2FE00223C21204600F0D5
:1012D000BDFE70222721204600F0B8FEFF22E22149
:1012E000204600F0B3FE10BD6133000810B504467F
:1012F00002222321204600F0A9FE04231E4A2A21AF
:10130000204600F065FE04231B4A3021204600F0F1
:101310005FFE30222121204600F098FE012222218A
:10132000204600F093FE12222521204600F08EFE7A
:1013300024222621204600F089FE0F22202120466B
:1013400000F084FE08223121204600F07FFE0122B9
:101350003D21204600F07AFE00223C21204600F08C
:1013600075FE70222721204600F070FEFF22E22148
:10137000204600F06BFE10BD9833000810B50446FF
:1013800002222321204600F061FE04231E4A2A2166
:10139000204600F01DFE04231B4A3021204600F0A9
:1013A00017FE30222121204600F050FE012222218A
:1013B000204600F04BFE28222521204600F046FE64
:1013C0000C222621204600F041FE0F22202120463B
:1013D00000F03CFE06223121204600F037FE0122BB
:1013E0003D21204600F032FE00223C21204600F044
:1013F0002DFE70222721204600F028FEFF22E22148
:10140000204600F023FE10BD8E33000810B50446C0
:1014100002222321204600F019FE04231E4A2A211D
:10142000204600F0D5FD04231B4A3021204600F061
:10143000CFFD30222121204600F008FE012222218A
:10144000204600F003FE16222521204600F0FEFD76
:1014500004222621204600F0F9FD0F2220212046FB
:1014600000F0F4FD08223121204600F0EFFD0122BA
:101470003D21204600F0EAFD00223C21204600F0FC
:10148000E5FD70222721204600F0E0FDFF22E22149
:10149000204600F0DBFD10BDA733000810B5044660
:1014A00002222321204600F0D1FD04231E4A2A21D6
:1014B000204600F08DFD04231B4A3021204600F019
:1014C00087FD30222121204600F0C0FD012222218B
:1014D000204600F0BBFD33222521204600F0B6FD5A
:1014E00004222621204600F0B1FD0F2220212046B3
:1014F00000F0ACFD09223121204600F0A7FD0122B9
:101500003D21204600F0A2FD00223C21204600F0B3
:101510009DFD70222721204600F098FDFF22E22148
:10152000204600F093FD10BD8433000810B504463A
:1015300002222321204600F089FD05231E4A2A218C
:10154000204600F045FD05231B4A3021204600F0CF
:101550003FFD3F222121204600F078FD012222217B
:10156000204600F073FD12222521204600F06EFD7A
:1015700004222621204600F069FD0F22202120466A
:1015800000F064FD0A223121204600F05FFD0122B7
:101590003D21204600F05AFD00223C21204600F06B
:1015A00055FD70222721204600F050FDFF22E22148
:1015B000204600F04BFD10BD5233000810B5044624
:1015C00002222321204600F041FD05231E4A2A2144
:1015D000204600F0FDFC05231B4A3021204600F088
:1015E000F7FC30222121204600F030FD012222218B
:1015F000204600F02BFD12222521204600F026FD7A
:1016000021222621204600F021FD0F222021204604
:1016100000F01CFD0A223121204600F017FD0022B7
:101620003D21204600F012FD01223C21204600F021
:101630000DFD70222721204600F008FDFF22E22147
:10164000204600F003FD10BD4333000810B50446EA
:1016500001222321204600F0F9FC05231E4A2A21FD
:10166000204600F0B5FC05231B4A3021204600F03F
:10167000AFFC30222121204600F0E8FC012222218B
:10168000204600F0E3FC19222521204600F0DEFC74
:1016900004222621204600F0D9FC0F2220212046DA
:1016A00000F0D4FC06223121204600F0CFFC0122BC
:1016B0003D21204600F0CAFC00223C21204600F0DB
:1016C000C5FC70222721204600F0C0FCFF22E22149
:1016D000204600F0BBFC10BD7033000810B5044676
:1016E0001CB900202749086003E0002025490C317F
:1016F000086001222321204600F0A8FC0323224A8F
:101700002A21204600F064FC0323204A3021204691
:1017100000F05EFC01222121204600F097FC01220E
:101720002221204600F092FC2A222521204600F0AA
:101730008DFC04222621204600F088FC0F22202167
:10174000204600F083FC06223D21204600F07EFC6E
:1017500001223C21204600F079FC702227212046FE
:1017600000F074FCFF22E221204600F06FFC1CB95F
:1017700001200449086003E0012002490C3108609F
:1017800010BD00009881214239330008343300082D
:1017900070B504460D461CB900203849086003E0C6
:1017A000002036490C310860142D5BD2DFE805F0CB
:1017B0000A0E12161A1E22262A2E32363A3E4246A9
:1017C0004A4E52562046FFF7F9FE4BE0204600F005
:1017D00097FA47E0204600F023FB43E02046FFF75E
:1017E000A5FE3FE0204600F0FBF93BE0204600F07C
:1017F000D7F837E02046FFF731FD33E0204600F010
:10180000A7F92FE0204600F0C3FA2BE02046FFF7AF
:101810001DFF27E0204600F033F823E0204600F0CB
:1018200027FA1FE0204600F073F81BE02046FFF780
:1018300035FE17E02046FFF709FF13E02046FFF7CB
:101840009DFD0FE0204600F03BF90BE02046FFF73E
:101850004DFD07E0204600F0EBF803E02046FFF7DF
:10186000D5FD00BF00BF1CB901200449086003E09A
:10187000012002490C31086070BD000098812142AE
:1018800010B5044602222321204600F0DFFB04238A
:101890001E4A2A21204600F09BFB04231B4A3021CC
:1018A000204600F095FB30222121204600F0CEFB9F
:1018B00001222221204600F0C9FB202225212046BA
:1018C00000F0C4FB20222621204600F0BFFB0F229F
:1018D0002021204600F0BAFB08223121204600F0EA
:1018E000B5FB01223D21204600F0B0FB00223C2147
:1018F000204600F0ABFB70222721204600F0A6FB1B
:10190000FF22E221204600F0A1FB10BD7533000844
:1019100010B5044602222321204600F097FB042341
:101920001E4A2A21204600F053FB04231B4A302183
:10193000204600F04DFB30222121204600F086FB9E
:1019400001222221204600F081FB1222252120467F
:1019500000F07CFB24222621204600F077FB0F229A
:101960002021204600F072FB0A223121204600F09F
:101970006DFB01223D21204600F068FB00223C2146
:10198000204600F063FB70222721204600F05EFB1A
:10199000FF22E221204600F059FB10BD7F330008F2
:1019A00010B5044602222321204600F04FFB0523F8
:1019B0001E4A2A21204600F00BFB05231B4A30213A
:1019C000204600F005FB30222121204600F03EFB9E
:1019D00001222221204600F039FB12222521204637
:1019E00000F034FB24222621204600F02FFB0F229A
:1019F0002021204600F02AFB0A223121204600F057
:101A000025FB01223D21204600F020FB00223C2145
:101A1000204600F01BFB70222721204600F016FB19
:101A2000FF22E221204600F011FB10BD5C330008CC
:101A300010B5044602222321204600F007FB0423B0
:101A40001E4A2A21204600F0C3FA04231B4A3021F3
:101A5000204600F0BDFA30222121204600F0F6FA9F
:101A600001222221204600F0F1FA142225212046ED
:101A700000F0ECFA04222621204600F0E7FA0F22BB
:101A80002021204600F0E2FA0A223121204600F00F
:101A9000DDFA01223D21204600F0D8FA00223C2147
:101AA000204600F0D3FA70222721204600F0CEFA1B
:101AB000FF22E221204600F0C9FA10BD9D33000844
:101AC00010B5044602222321204600F0BFFA042369
:101AD0001E4A2A21204600F07BFA04231B4A3021AB
:101AE000204600F075FA30222121204600F0AEFA9F
:101AF00001222221204600F0A9FA122225212046A7
:101B000000F0A4FA24222621204600F09FFA0F229A
:101B10002021204600F09AFA08223121204600F0C8
:101B200095FA01223D21204600F090FA00223C2146
:101B3000204600F08BFA70222721204600F086FA1A
:101B4000FF22E221204600F081FA10BD9333000805
:101B500010B5044601222321204600F077FA052320
:101B60001E4A2A21204600F033FA05231B4A302161
:101B7000204600F02DFA30222121204600F066FA9E
:101B800001222221204600F061FA10222521204660
:101B900000F05CFA04222621204600F057FA0F22BA
:101BA0002021204600F052FA06223121204600F082
:101BB0004DFA01223D21204600F048FA00223C2146
:101BC000204600F043FA70222721204600F03EFA1A
:101BD000FF22E221204600F039FA10BD66330008EA
:101BE00010B5044602222321204600F02FFA0523D7
:101BF0001E4A2A21204600F0EBF905231B4A30211A
:101C0000204600F0E5F930222121204600F01EFA9E
:101C100001222221204600F019FA12222521204615
:101C200000F014FA24222621204600F00FFA0F2299
:101C30002021204600F00AFA08223121204600F037
:101C400005FA01223D21204600F000FA00223C2145
:101C5000204600F0FBF970222721204600F0F6F91B
:101C6000FF22E221204600F0F1F910BD57330008B1
:101C700010B5044602222321204600F0E7F9042390
:101C80001E4A2A21204600F0A3F904231B4A3021D2
:101C9000204600F09DF930222121204600F0D6F99F
:101CA00001222221204600F0D1F91C2225212046C4
:101CB00000F0CCF924222621204600F0C7F90F229B
:101CC0002021204600F0C2F908223121204600F0F0
:101CD000BDF901223D21204600F0B8F900223C2147
:101CE000204600F0B3F970222721204600F0AEF91B
:101CF000FF22E221204600F0A9F910BD7A33000846
:101D000010B5044603222321204600F09FF9052345
:101D10001E4A2A21204600F05BF905231B4A302188
:101D2000204600F055F93F222121204600F08EF98F
:101D30003F222221204600F089F928222521204631
:101D400000F084F904222621204600F07FF90B22BE
:101D50002021204600F07AF90A223121204600F0A5
:101D600075F901223D21204600F070F900223C2146
:101D7000204600F06BF970222721204600F066F91A
:101D8000FF22E221204600F061F910BD483300082F
:101D900010B5044601222321204600F057F9032301
:101DA0001E4A2A21204600F013F903231B4A302142
:101DB000204600F00DF930222121204600F046F99E
:101DC00001222221204600F041F92A222521204625
:101DD00000F03CF904222621204600F037F90F22BA
:101DE0002021204600F032F907223121204600F060
:101DF0002DF900223D21204600F028F901223C2146
:101E0000204600F023F970222721204600F01EF919
:101E1000FF22E221204600F019F910BD6B330008C3
:101E200010B5044603222321204600F00FF90523B4
:101E30001E4A2A21204600F0CBF805231B4A3021F8
:101E4000204600F0C5F830222121204600F0FEF89F
:101E500001222221204600F0F9F8102225212046F7
:101E600000F0F4F804222621204600F0EFF80F22BB
:101E70002021204600F0EAF80A223121204600F015
:101E8000E5F801223D21204600F0E0F800223C2147
:101E9000204600F0DBF870222721204600F0D6F81B
:101EA000FF22E221204600F0D1F810BD4D3300089A
:101EB0002DE9F0478046894615461E46B8F1000FC9
:101EC00016D10020174908604946404600F024FB1F
:101ED0000746002406E0FF21404600F01DFB285580
:101EE000601CC4B2B442F6DB01200E49086015E064
:101EF00000200D4908604946404600F00DFB0746AA
:101F0000002406E0FF21404600F006FB2855601C37
:101F1000C4B2B442F6DB0120034908603846BDE88C
:101F2000F087000090012142B081214270B5054642
:101F30000E4685B90020114908603146284600F058
:101F4000EBFAFF21284600F0E7FA044601200C498D
:101F5000C1F890010FE000200A4908603146284688
:101F600000F0DAFAFF21284600F0D6FA04460120F4
:101F70000549C1F8B001204670BD00009001214222
:101F800000002142B08121420080214270B5064606
:101F90000D461021304600F013FB07213046FFF7B5
:101FA000C5FF044622462721304600F04FF804F0D2
:101FB000400050B10A232A4661213046FFF778FFDE
:101FC000FF22E221304600F041F8204670BD0000BB
:101FD0002DE9F0478046894615461E46B8F1000FA8
:101FE00016D10020174908604946404600F094FA8F
:101FF0000746002406E015F8011B404600F08CFA65
:10200000601CC4B2B442F6DB01200E49086015E042
:1020100000200D4908604946404600F07DFA074619
:10202000002406E015F8011B404600F075FA601C1C
:10203000C4B2B442F6DB0120034908603846BDE86B
:10204000F087000090012142B08121422DE9F0414A
:1020500004460E46154684B90020114908603146F1
:10206000204600F059FA07462946204600F054FA67
:1020700001200C49C1F890010FE000200A490860D6
:102080003146204600F048FA07462946204600F02F
:1020900043FA01200549C1F8B0013846BDE8F08196
:1020A0009001214200002142B08121420080214262
:1020B00008B54FF4C06000F071F826208DF80000DC
:1020C00001208DF8010002208DF8020001208DF81A
:1020D0000300684600F02AF827208DF80000012050
:1020E0008DF801008DF802008DF80300684600F0BD
:1020F0001DF825208DF8000000208DF8010001203A
:102100008DF802008DF80300684600F00FF81D20DE
:102110008DF8000000208DF801008DF802000120EC
:102120008DF80300684600F001F808BD70B5002185
:1021300000230F22C47804B3154C246804F4E0642F
:10214000C4F5E064210AC1F10403CA40447804FAEA
:1021500003F184781440214309010E4C0678A155FF
:10216000047804F01F050124AC4005786D11AD0022
:1021700005F1E025C5F8004109E0047804F01F05E9
:102180000124AC40044D0678761145F8264070BD18
:102190000CED00E000E400E080E100E002490143D2
:1021A000024A1160704700000000FA050CED00E0E3
:1021B0007047000029B1064AD2690243044BDA6134
:1021C00004E0034AD2698243014BDA6170470000A0
:1021D0000010024029B1064A92690243044B9A61F9
:1021E00004E0034A92698243014B9A617047000000
:1021F0000010024070B5012144F20D00FFF7EAFF24
:1022000001210220FFF7D6FF042000F013FB124942
:10221000B1F1807F00D31DE021F07F40401E4FF0E0
:10222000E022506150170F22002807DA13071D0E15
:102230000A4B00F00F04241F1D5503E013071C0E6A
:10224000074B1C5400BF00204FF0E0229061072094
:10225000106100BF70BD000080A9030018ED00E010
:1022600000E400E070B500210023002400220025D6
:102270002C4E766806F00C0121B1042905D00829FE
:1022800021D105E0284E066020E0274E06601DE0C3
:10229000244E766806F47013224E766806F4803475
:1022A000022606EB93431CB9204E5E43066009E00C
:1022B0001C4E7668C6F34046751C1B4EB6FBF5F601
:1022C0005E43066002E0184E066000BF00BF154E78
:1022D000766806F0F0010909154E725C0668D64072
:1022E0004660104E766806F4E061090A104E725C92
:1022F0004668D64086600B4E766806F46051C90A7F
:102300000B4E725C4668D640C660064E766806F490
:102310004041890B074E725CC668B6FBF2F6066157
:1023200070BD00000010024000127A0000093D005C
:102330008E0000209E00002010B586B000241421DD
:1023400001A8FDF718FF0A2201A9084800F012F8B9
:1023500000BF07E001A810F81400054A02F81400B5
:10236000601CC4B20A2CF5DB06B010BD00000308E7
:102370004805002070B504460D461646002300BFF0
:1023800007E02046FEF76EFE25F81300A41C581C3B
:10239000C3B2B342F5DB70BD00B587B0012141F295
:1023A0000500FFF717FFE020ADF8180018208DF8A2
:1023B0001B0003208DF81A0006A91648FEF7C3FD7E
:1023C000E0211448FEF74CFE0020ADF804004FF465
:1023D0008270ADF806000020ADF80800ADF80A00E4
:1023E000ADF80C004FF40070ADF80E001820ADF8F9
:1023F00010000020ADF812000720ADF8140001A96C
:10240000054800F06BF80121034800F04DF807B0D3
:1024100000BD0000000801400030014000B587B059
:1024200001218803FFF7C6FE01210920FFF7D2FE34
:102430004FF46040ADF8180018208DF81B00032001
:102440008DF81A0006A91648FEF77DFD4FF460418D
:102450001348FEF705FE0020ADF804004FF482702B
:10246000ADF806000020ADF80800ADF80A00ADF8A0
:102470000C004FF40070ADF80E001820ADF81000FD
:102480000020ADF812000720ADF8140001A905489E
:1024900000F024F80121034800F006F807B000BD61
:1024A000000C01400038004021B1028842F0400297
:1024B000028004E002884FF6BF731A400280704722
:1024C0000246002013890B400BB1012000E00020E0
:1024D00070470146888970478181704710B5002296
:1024E000028802F441520B884C8823438C88234392
:1024F000CC8823430C8923434C8923438C89234371
:10250000CC8923431A430280838B4FF2FF7423400C
:1025100083830B8A038210BD2DE9F04106460F46E6
:1025200026BB06E0601CC4B2C82C02DB0020BDE85C
:10253000F08102212048FFF7C3FF0028F2D039467E
:102540001D48FFF7C9FF002405E0601CC4B2C82C79
:1025500001DB0020EBE701211748FFF7B1FF00285E
:10256000F3D01548FFF7B5FFC5B222E005E0601CC7
:10257000C4B2C82C01DB0020D9E702210F48FFF7C5
:102580009FFF0028F3D039460C48FFF7A5FF002431
:1025900005E0601CC4B2C82C01DB0020C7E70121A4
:1025A0000648FFF78DFF0028F3D00448FFF791FF9E
:1025B000C5B22846BBE700000030014000380040AB
:1025C00070B505460C467DB90F4800884FF6C771B7
:1025D00008400D49088008460088204308800121F2
:1025E0000A48FFF761FF0EE0084800884FF6C77100
:1025F00008400649088008460088204308800121D9
:102600000248FFF751FF70BD003001400038004024
:10261000704770B504460D4629462046FEF754FC27
:1026200070BD000010B586B00024142101A8FDF78C
:10263000A2FD00BF07E00B4830F8140001A921F803
:102640001400601CC4B20A2CF5DB074800F0EAF85D
:102650000A2201A9044800F009F800F07AFC06B04B
:1026600010BD000034050020000003082DE9F041F2
:1026700005460F461646002400BF07E037F8141041
:102680002846FFF7C6FFAD1C601CC4B2B442F5DBA0
:10269000BDE8F08170B504460D46034A2946204640
:1026A00000F028F870BD00000038014010B5044665
:1026B0000249204600F00EF810BD00000044004022
:1026C00010B504460249204600F02DF810BD000068
:1026D0000044004070B504460D4600BF80212846E6
:1026E00000F064FB0028F9D02146284600F02BFCBE
:1026F000012070BD2DE9F04104460D46164614B97F
:102700000120BDE8F0810AE014F8017B314638462B
:10271000FFF7E0FF08B90020F3E7681E85B2002D3F
:10272000F2D10120EDE770B504460E460CB9012048
:1027300070BD11E014F8015B0A2D06D131460D2061
:10274000FFF7C8FF08B90020F2E731462846FFF737
:10275000C1FF08B90020EBE720780028EAD101206A
:10276000E6E710B500F002F810BD00000CB500203F
:10277000019000902A48006840F4803028490860A1
:1027800000BF2748006800F4003000900198401C0A
:102790000190009818B90198B0F5A06FF1D12048C8
:1027A000006800F4003010B10120009001E000202A
:1027B00000900098012831D11948406818494860B4
:1027C00008464068486008464068486008464068D7
:1027D00020F47C1048600846406840F49810486037
:1027E0000846006840F08070086000BF0C48006830
:1027F00000F000700028F9D00948406820F003007C
:10280000074948600846406840F00200486000BF41
:102810000348406800F00C000828F9D10CBD000006
:102820000010024010B50446FEF76EFB2046FEF78E
:1028300001FB10BD042808D14FF0E021096941F0E7
:1028400004014FF0E022116107E04FF0E021096937
:1028500021F004014FF0E022116170477047000041
:1028600010B51448006840F001001249086008469D
:102870004068114908400F494860084600680F4900
:1028800008400C4908600846006820F48020086071
:102890000846406820F4FE0048604FF41F0088603E
:1028A0000020C862FFF75DFF4FF000600449086038
:1028B00010BD0000001002400000FFF8FFFFF6FE10
:1028C00008ED00E010B50121204800F07EF8002856
:1028D0003AD001211D4800F069F81D480088401CCD
:1028E0001B4908801B480088401C1A4908801A4868
:1028F0000088401C1849088018480078C0B14FF47F
:1029000000711748FEF7ACFB16480088401C1549BB
:10291000088008460088B0F5C87F09DB4FF40071D5
:102920000F48FEF79BFB00200E4908800B490870FA
:102930000948008841F28831884202D100200649C6
:10294000088001200849087010BD00000004004004
:102950002600002038000020280000202B00002046
:10296000001001402C0000202A0000203EB5054642
:102970000C4601210220FFF71DFCADF80450ADF814
:1029800000400020ADF80600ADF802006946064898
:1029900000F036F801221146034800F027F8012123
:1029A000014800F006F83EBD00040040CA43028220
:1029B000704721B1028842F00102028004E00288DF
:1029C0004FF6FE731A400280704730B50246002071
:1029D00000230024158A05EA0103958905EA01040C
:1029E00013B10CB1012000E0002030BD1AB1838981
:1029F0000B43838102E083898B438381704700000E
:102A0000002202881D4B98420ED01D4B98420BD0DD
:102A1000B0F1804F08D01B4B984205D01A4B98421A
:102A200002D01A4B984204D14FF68F731A404B884C
:102A30001A43174B984207D0164B984204D04FF6D2
:102A4000FF431A40CB881A4302808B8883850B880A
:102A500003850A4B98420BD0094B984208D00E4B85
:102A6000984205D00D4B984202D00D4B984201D1AF
:102A70000B7A03860123838270470000002C0140FB
:102A8000003401400004004000080040000C0040F9
:102A9000001000400014004000400140004401408C
:102AA0000048014010B540F22551124800F08BF962
:102AB00088B140F225510F4800F0CFF80D4800F0E2
:102AC0003DFAC4B20C480D49097844540B480078CB
:102AD000401C0A4908700821064800F067F90128DF
:102AE00006D10821034800F0AFF8024800F026FAAA
:102AF00010BD0000003801400C0100200300002040
:102B000010B540F22551124800F05DF988B140F24D
:102B100025510F4800F0A1F80D4800F00FFAC4B29B
:102B20000C480D49097844540B480078401C0A4968
:102B300008700821064800F039F9012806D108215B
:102B4000034800F081F8024800F0F8F910BD0000D9
:102B500000440040F40400208B00002010B586B033
:102B6000044601210520FFF735FB01214804FFF74A
:102B700021FB0420ADF8140003208DF81600182066
:102B80008DF8170005A91548FEF7DDF90820ADF806
:102B9000140004208DF8170005A91048FEF7D3F99A
:102BA00001940020ADF80800ADF80A00ADF80C0063
:102BB000ADF810000C20ADF80E0001A9084800F097
:102BC00051F9012240F22551054800F026F9012172
:102BD000034800F051F806B010BD000000080140A5
:102BE0000044004010B540F22551144800F0EBF8C5
:102BF000B0B140F22551114800F02FF80F4800F015
:102C00009DF9C4B20E480F49097844540D48007824
:102C1000401C0C4908700846007800F00F0008704E
:102C20000821064800F0C2F8012806D1082103480F
:102C300000F00AF8014800F081F910BD004800409A
:102C4000D40100200900002001F40072B2F5007FD9
:102C500000D100BFCA430280704710B50022002394
:102C600040F66A14A14200D100BF0A120124944028
:102C7000A3B2DC43048010BD21B1828942F400522A
:102C8000828104E082894DF6FF731A408281704789
:102C900000B585B0012144F20400FFF79BFA4FF420
:102CA0000070ADF8000003208DF8020018208DF8A8
:102CB000030069463948FEF746F94FF48060ADF8E5
:102CC000000004208DF8030069463448FEF73BF904
:102CD0004FF4164001900020ADF80800ADF80A004E
:102CE000ADF80C00ADF810000C20ADF80E0001A9F5
:102CF0002B4800F0B7F8012240F22551284800F097
:102D00008CF801212648FFF7B7FF01218804FFF75F
:102D100051FA01210820FFF75DFA4FF48060ADF809
:102D2000000003208DF8020018208DF8030069468A
:102D30001C48FEF708F94FF40060ADF800000420CD
:102D40008DF8030069461748FEF7FDF84FF49650DA
:102D500001900020ADF80800ADF80A00ADF80C00B5
:102D6000ADF810000C20ADF80E0001A90E4800F0DF
:102D700079F801A90C4800F075F8012240F22551BC
:102D8000094800F04AF801210748FFF775FF402184
:102D90000348FFF759FF05B000BD000000080140DF
:102DA00000380140000C014000480040024600206D
:102DB000B1F5007F00D100BF13880B400BB101209B
:102DC00000E00020704770B5024600240023002573
:102DD000002040F66A16B14200D100BFC1F342158F
:102DE00001F01F03012606FA03F3012D02D1968993
:102DF000334006E0022D02D1168A334001E0968A64
:102E000033400C12012606FA04F41688344013B13C
:102E10000CB1012000E0002070BDF0B50346002495
:102E200000260025002040F66A17B94200D100BFF5
:102E30001846C1F3421401F01F06012707FA06F5F0
:102E4000012C01D10C3004E0022C01D1103000E043
:102E500014301AB107682F43076002E00768AF43D8
:102E60000760F0BD2DE9F04786B005460E46002408
:102E7000A24600BFA1460027B08900B100BF2F467F
:102E80002C8A4CF6FF700440F08804432C82AC89F5
:102E90004EF6F3100440B088318908437189084325
:102EA0000443AC81AC8A4FF6FF400440B089044330
:102EB000AC8201A8FFF7D6F91F48874202D1DDF89E
:102EC00010A001E0DDF80CA0A88900F4004040B19A
:102ED0000AEBCA0000EB0A1031684900B0FBF1F8B8
:102EE00007E00AEBCA0000EB0A1031688900B0FB6A
:102EF000F1F86420B8FBF0F004012009642101FB23
:102F00001089A88900F4004040B1322000EBC900CC
:102F1000B0FBF1F000F00700044308E0322000EBC2
:102F200009106421B0FBF1F000F00F0004432C8184
:102F300006B0BDE8F08700000038014001468888EF
:102F4000C0F308007047C1F308028280704700BFD9
:102F5000FEE710B5FDF7AEFF10BD0000014A0249C3
:102F600000F013B8D92F0008A400002002E008C820
:102F7000121F08C1002AFAD170477047002001E0F3
:102F800001C1121F002AFBD170472DE9F0411646FE
:102F90000F460446002503E03946B047641C6D1C0B
:102FA00020780028F8D12846BDE8F08110B5024607
:102FB0000BE0C82007E0122101E04B1E99B2002966
:102FC000FBDC431E98B20028F5DC131EA2F10104BD
:102FD000A2B2EED110BD000070B504460D46E0B2BD
:102FE0000549088000BF40210348001FFFF7DEFEAF
:102FF0000028F8D0204670BD0438014008B50121F2
:103000001020FFF7E7F80120ADF8000010208DF840
:10301000030003208DF8020069460D48FDF793FF79
:1030200001210B48FEF71CF84FF40070ADF80000CA
:1030300010208DF8030003208DF802006946044833
:10304000FDF781FF4FF400710148FEF707F808BD56
:1030500000100140FFF7CEF8FFF72AF840F2712187
:103060000420FEF721F8FEF71BF841F61F41092066
:10307000FFF77CFCFFF7C2FFFFF70AFE4FF4E130D9
:10308000FFF76CFDFEF76CF8FEF70AF802E04DA0C2
:10309000FFF764FF0120FEF737F80028F7D1FDF7AE
:1030A0000DFEFDF7FDFF4B480068C0434A49C1F8DB
:1030B0008001C820FFF77AFF4748D0F88001C0435D
:1030C0004549C1F88001062144A0FDF798FE45A0BE
:1030D000FFF7F6FAFDF7E4FF43A0FFF73FFF0120FB
:1030E000FEF7FCFAFFF728F94848007848490870CD
:1030F0000846007814285BD2DFE800F00A0E1216AA
:103100001A1E22262A2E32363A3E42464A4E52563F
:1031100040A0FFF723FF4BE041A0FFF71FFF47E070
:1031200042A0FFF71BFF43E043A0FFF717FF3FE07C
:1031300044A0FFF713FF3BE045A0FFF70FFF37E088
:1031400047A0FFF70BFF33E048A0FFF707FF2FE092
:103150004AA0FFF703FF2BE04BA0FFF7FFFE27E09D
:103160004CA0FFF7FBFE23E04DA0FFF7F7FE1FE0AA
:103170004FA0FFF7F3FE1BE052A0FFF7EFFE17E0B2
:1031800054A0FFF7EBFE13E056A0FFF7E7FE0FE0B9
:1031900058A0FFF7E3FE0BE05AA0FFF7DFFE07E0C1
:1031A0005CA0FFF7DBFE03E05EA0FFF7D7FE00BFE9
:1031B00000BF3220FFF7FAFE03E0FDF71BF8FDF732
:1031C0007BFAFAE754686520322E34472045727244
:1031D0006F722100800122420000224231323334DA
:1031E000353600000A0000000A5043B6D4C2EBC8CE
:1031F000EDBCFECDA8D3C3B0E6B1BE56322E322D03
:1032000032303138303931330A00000048050020AF
:1032100030000020BDADCEF7D0ADD2E90D0A0000E0
:10322000CCECB2A8D0ADD2E90D0A0000D4C6C4CF10
:10323000D0ADD2E90D0A0000B9F3D6DDD0ADD2E9A8
:103240000D0A0000CBC4B4A8D0ADD2E90D0A00002D
:10325000C4DAC3C9B9C5D0ADD2E90D0A0000000077
:10326000B0B2BBD5D0ADD2E90D0A0000C9BDCEF7D2
:10327000F6CEC5B5D0ADD2E90D0A000056434F4D8C
:10328000B2E2CAD40D0A0000C1C9C4FEB5E7D0C578
:103290000D0A0000C1C9C4FED2C6B6AF0D0A0000B7
:1032A0005470D7A8D3C3D0ADD2E90D0A00000000F6
:1032B000C4DAC3C9B9C5D2C6B6AFD0ADD2E90D0A1A
:1032C00000000000B9E3CEF7D2C6B6AFD0ADD2E968
:1032D0000D0A0000CBC4B4A8B5E7D0C5D0ADD2E983
:1032E0000D0A0000B8A3BDA8D5E6D7C6D0ADD2E977
:1032F0000D0A0000CBD5D6DDC4BEC0BCD0ADD2E92E
:103300000D0A0000D6D8C7ECD2C6B6AFD0ADD2E910
:103310000D0A0000C9BDCEF7D2C6B6AFD0ADD2E916
:103320000D0A0000B8CACBE0D2C6B6AFD0ADD2E924
:103330000D0A0000344310100134431010013320F3
:103340000D547933200D54793443101001011010BD
:1033500043343223ABBA013412BBAA01341286754E
:10336000014656431000346E4610013443101001DC
:10337000862C95010136E4A7BC014218BAE8013455
:103380001286750133200D5400862C9500005A4595
:103390004E4B00AABB1234003412BBAA00254310C6
:1033A0001200E77EE300004222B6E900CC330008B9
:1033B00000000020A80000006C2F000874340008F2
:1033C000A8000020585F00007C2F000800000000CB
:1033D0000000000000000000D1D1E0D0000000009B
:1033E000D2D2000000000000000000000000000039
:1033F00000000000000000000000000000000000CD
:1034000000000000000000000000000000000000BC
:103410000000000031323334353637383931323339
:103420003435363738390000000000000000000055
:103430000000000031323334353637383931323319
:103440003435363738390000000000000000000035
:103450000000000000000000000000000000010269
:103460000304010203040607080902040608000019
:043470000000000058
:0400000508000131BD
:00000001FF
